:020000000126D7
:03000300020803ED
:03000B0002080BDD
:03001300020813CD
:03001B0002081BBD
:1000230002082375817053D0E775A80075C7AA75B8
:10003300C75575C612907F8074007E13F0A3DEFC53
:10004300907F907400F0A37408F0907F927470F026
:1000530074FA907F93F0412B8E7E8F7F20B3FD7EC9
:1000630047DEFE7F08A2B3137E2DDEFE00DFF6C35C
:10007300AF7FAE7E228E7E8F7FC2B57E2FDEFE7F68
:10008300081392B57E2DDEFE00DFF6D2B57E2FDE9D
:10009300FEAF7FAE7E22046A000000000003120060
:1000A300B638303531206D6F6E69746F72205631FA
:1000B3002E320075C7AA75C75575C612C0E0740104
:1000C300C0A8C2AFC083C082907F80F0A37400F049
:1000D300A3E5D0F0A3D0E0F0A3D0E0F0A3D0E0F00C
:1000E300A3D0E0F0A3E5F0F0A371A0907F80E0F847
:1000F300D0E0F9D0E0B8010524FD400119907F90CC
:10010300F0A3E9F0A3E581F0412B75C7AA75C755A4
:1001130075C612907F93115B40F0B4F70040EBF08B
:10012300A3115B40E5B46B0050E0F0A36009FE113E
:100133005B40D7F0A3DEF8115B40CFFD718D2D70CE
:10014300C9907F93E0FEA3E0CEA3B4FF022184B461
:10015300FE0221A2B4FD0221D0B4FC02412BB4FB68
:1001630002415BB4FA02419EB4F90241DDB4F802E4
:10017300611CB4F702613F74F0907F93F0740161E6
:1001830069907F94741DF0A3FE7F00A882A98390D9
:100193000099EF930F88828983F0A3DEEE6175A344
:1001A300E0F8A3E0F9A3E0FE907F94F0A3601CAA1B
:1001B30082AB8388828983B90003E68001E0A3A828
:1001C30082A9838A828B83F0A3DEE46175A3E0F8BE
:1001D300A3E0F9A3EE24FD6047FEFFE0AA82AB8310
:1001E30088828983B90003F68001F0A3A882A983DA
:1001F3008A828B83A3DEE4907F96E0F8A3E0F9A3E1
:10020300E0FEAA82AB8388828983B90003E680017A
:10021300E06E7010A3A882A9838A828B83A3DFE098
:10022300740080027401616975C7AA75C75575C6E4
:1002330012907F807413FEA882A983907F94F0A309
:10024300AA82AB8388828983E0A3A882A9838A8256
:100253008B83F0A3DEEA6175EE603EA3A3E054183E
:10026300F5F065D054186011907F9D71B953D0E7B4
:10027300E5F042D0907F9D71A07880797F907F9444
:10028300E0FEA3E0A3AA82AB8388828983F0A3A8BC
:1002930082A9838A828B83DEEA412B907F92E0F5E9
:1002A30081907F8871B9E0C0E0A3E0C0E0907F85D2
:1002B300E0C0E0A3E0C0E0A3E0F5F0A3907F82E01C
:1002C300F5D0A3E0C0E0A3E0F583D082D0E0D0A8CE
:1002D30075C7AA75C75575C68022EE6032AA82AB70
:1002E30083AC82AD838A828B83A3E0F8A3E0F9A376
:1002F300E0FFA3AA82AB8388828983E0F8EFF0E072
:100303008C828D836F7008E8F0A31E1E1EDED2E57B
:1003130082246B907F94F06175E0F874E5F0A3E8B4
:10032300F0A37422F075C7AA75C75575C680127FEE
:100333009575C7AA75C75575C6126169E0F8A3A379
:10034300E0F974F5F0A3E8F0A37422F0E975C7AA05
:1003530075C75575C680127F9775C7AA75C755753A
:10036300C61274006169F8907F947401F0A3E8F0F9
:100373008000718D64FF04F0907F94E02403FE906D
:100383007F93E01178A3DEFA210D907F94E024029D
:10039300FE907F937F00E02FFFA3DEFA22E8F0A315
:1003A300E9F0A3EAF0A3EBF0A3ECF0A3EDF0A3EEE6
:1003B300F0A3EFF0A322E0F8A3E0F9A3E0FAA3E0AF
:0F03C300FBA3E0FCA3E0FDA3E0FEA3E0FFA32269
:00002601D9
